:1042DC0000010C01010502011E030A9604013205BE
:1042EC00040406006407010108000009015A0E01CC
:1042FC00010F000112006413010114013C1501FAB5
:10430C001664FA17FFFF1D00072000072400022780
:10431C0001012F013C30030332010335FFFF36034B
:10432C00073CFFFF3DFFFF180002191E461A000252
:10433C001B00022D32C82E0001FAFAFA18000019DF
:10434C00FFFF1A00001B00002D32C82E0001FAFAE4
:10435C00FA18000019FFFF1A00001B00002DFFFFC8
:06436C002EFFFFFAFAFA31
:10004800900786E0FEA3E0FF7457BE0010D39F40E0
:100058000C9042DC12001EE493F599804C90001439
:10006800E0D394044014900786E0FEA3E0FF90429A
:10007800DC12001EE493F599802F900014E0D394CD
:10008800034014900786E0FEA3E0FF9042F11200BF
:100098001EE493F5998012900786E0FEA3E0FF9096
:1000A800430612001EE493F59990078612000E90FD
:1000B8000786E0FEA3E0FF746C6F4E7003751300B3
:1000C80022900072E0B401087402900072F0D20F1E
:1000D80090013AE090002AF090013BE090002BF06C
:1000E80090013CE090002CF0A20DB3401690013A2C
:1000F800E0700C90013BE0700690013CE0600280EB
:1001080002C20D90013AE0B4300F90013BE0B447D1
:100118000890013CE0643B60028004D20E8002C279
:100128000EE558B40102800302024B900057E0F537
:1001380066900062E0F568900063E0F569900074ED
:10014800E0F56A90007AE0900029F090007CE0F5F4
:100158006590007DE0F567900080E0F5649000818F
:10016800E0F563900090E0900041F0900091E090FD
:100178000042F0900092E0900043F0900093E090ED
:100188000044F0900094E0900045F0900095E090D5
:100198000046F0900096E0900047F0900097E090BD
:1001A8000048F0900099E0900033F090009AE090B9
:1001B8000034F090009BE0900035F090009CE090B7
:1001C8000036F0900079E0B4011790000A740FF03F
:1001D800A374FFF090000CE4F0A3F074029000798F
:1001E800F0900079E0B4035990000CE0FEA3E0FF22
:1001F80090000AE0FCA3E0FD12000374101243F122
:1002080074081243E3EF900026F0EF700674FF9035
:100218000026F07400900079F090000BE090002721
:10022800F090000AE0900028F0900026E0900789FE
:10023800F0900027E090078AF0900028E090078B64
:10024800F0803F900081E07006755801756300A248
:100258000DB3402E90013AE090002AF090013BE067
:1002680090002BF090013CE090002CF090002AE0E8
:10027800700C90002BE0700690002CE06002800269
:10028800C20DE5667003756602E56870037568025D
:100298007E817F99E5668E048F05FF1243D38C39E2
:1002A8008D3AE56975F0FAA4FFAEF0E5688E048F23
:1002B80005FF1243D38C3D8D3E90004FE0F56090D2
:1002C800004DE0FE900069E0B5061890004CE0FE95
:1002D800900068E0B5060C90004BE0FE900059E0F5
:1002E8006E606F900069E07006900068E0600674C8
:1002F80000900059F0900069E0B402089000497439
:1003080001F08005900049E4F0900068E0B402082C
:1003180090004A7401F0800590004AE4F09000686B
:10032800E0600690004AE060028005756004800382
:10033800756005E559B55802D20F900068E0900045
:100348004CF0900069E090004DF0900059E090006A
:100358004BF0740190009EF0740090009FF07401BF
:100368009000A0F074009000A1F074009000A2F03A
:1003780074009000A3F074009000A4F07401900041
:10038800A5F074009000A6F074009000A7F0740027
:100398009000A8F074009000A9F074009000AAF0F2
:1003A80074009000ABF074019000ACF07400900001
:1003B800ADF074019000AEF074009000AFF07400DE
:1003C8009000B0F074009000B1F074009000B2F0AA
:1003D8007401900362F07400900363F0740090035A
:1003E80064F07400900365F07400900366F0740084
:1003F800900367F07400900368F074019003A2F012
:1004080074019003A3F074009003A4F074009003A7
:10041800A5F074009003A6F074009003A7F0740090
:100428009003A8F074009003E2F074019003E3F0E5
:1004380074009003E4F074009003E5F074009003F6
:10044800E6F074009003E7F074009003E8F074009D
:10045800900422F07400900423F07401900424F0B6
:100468007400900425F07400900426F07400900441
:1004780027F07400900428F07400900462F074006F
:10048800900463F07400900464F07401900465F0C3
:100498007400900466F07400900467F0740090048F
:1004A80068F022E5B554F7F5B5E5B554FDF5B5C2E4
:1004B80093C294C291C292C207C208E5B554FBF533
:1004C800B5755105E55104F55290004FE0F560907F
:1004D8000025E4F0C20CE5B554FEF5B522750A0016
:1004E800750900AE09AF0A7457BE00039F50030296
:1004F80005A29042DC12001EE49390004E124409BB
:100508000FBF00010EE0FC9042DC12001EECFEE47E
:1005180093FFEEC39F5026AE09AF0A0FBF00010E2E
:100528009042DC12001EAE09AF0AE493FC9042DC54
:1005380012001EE49390004E124409ECF0AE09AF8D
:100548000A9042DC12001EE49390004E124409E027
:10055800FC9042DE12001EECFCE493FDECD39D40BF
:10056800199042DE12001EE493FC9042DC12001E39
:10057800E49390004E124409ECF0AE09AF0A7402FD
:100588002FFF50010E8E098F0A780A740126F65043
:100598000418E436F640030204EB22750A007509D4
:1005A80000AE09AF0A7415BE00039F50030206701F
:1005B80090433312001EE49390004E1244090FBF7B
:1005C80000010EE0FC90433312001EECFEE493FFA2
:1005D800EEC39F5026AE09AF0A0FBF00010E90432D
:1005E8003312001EAE09AF0AE493FC9043331200A5
:1005F8001EE49390004E124409ECF0AE09AF0A9045
:10060800433312001EE49390004E124409E0FC901C
:10061800433512001EECFCE493FDECD39D40199089
:10062800433512001EE493FC90433312001EE493FA
:1006380090004E124409ECF0AE09AF0A740F6F4EE9
:100648007006750A15750900AE09AF0A74022FFF06
:1006580050010E8E098F0A780A740126F650041884
:10066800E436F640030205A922750A00750900AEB2
:1006780009AF0A7415BE00039F500302073E90435A
:100688004812001EE49390004E1244090FBF000167
:100698000EE0FC90434812001EECFEE493FFEEC30C
:1006A8009F5026AE09AF0A0FBF00010E90434812B3
:1006B800001EAE09AF0AE493FC90434812001EE402
:1006C8009390004E124409ECF0AE09AF0A904348EB
:1006D80012001EE49390004E124409E0FC90434A35
:1006E80012001EECFCE493FDECD39D401990434AA4
:1006F80012001EE493FC90434812001EE4939000FD
:100708004E124409ECF0AE09AF0A740F6F4E700632
:10071800750A15750900AE09AF0A74022FFF50015A
:100728000E8E098F0A780A740126F6500418E436EA
:10073800F6400302067722750A00750900AE09AF74
:100748000A7415BE00039F500302080C90435D1203
:10075800001EE49390004E1244090FBF00010EE002
:10076800FC90435D12001EECFEE493FFEEC39F5025
:1007780026AE09AF0A0FBF00010E90435D12001E9E
:10078800AE09AF0AE493FC90435D12001EE4939017
:10079800004E124409ECF0AE09AF0A90435D120016
:1007A8001EE49390004E124409E0FC90435F12004F
:1007B8001EECFCE493FDECD39D401990435F1200BE
:1007C8001EE493FC90435D12001EE49390004E12C9
:1007D8004409ECF0AE09AF0A740F6F4E7006750A43
:1007E80015750900AE09AF0A74022FFF50010E8E6D
:1007F800098F0A780A740126F6500418E436F64080
:100808000302074522054D22054C22054EC2CF2280
:1008180090F800E4936406600280FE75840175A771
:100828000075FF80900788E4F075C91075A70F75EB
:10083800A1C775A70075D90075CEFF75A70F75F10B
:10084800FE75F2FF75F33775F47875A4BA75A5FFD0
:1008580075A60775AE0075AFFF75D48175D5FF75A0
:10086800D6FF75D7FFC296C295C2A0C297C291C2E1
:1008780093C294E5B554DFF5B5E5B554EFF5B5E5A4
:10088800B5547FF5B5E5B554F7F5B5E5B554FDF5BF
:10089800B575A70075A20175A14775F80975BC0162
:1008A80075BE0475BD6C75BE0775BDA075BE0875AF
:1008B800BD0175BC0075BB1875BC2075BA0875E814
:1008C8008075D11375A70F75E10575E20075C740EE
:1008D800759700759780740A1243C37597C0E5979A
:1008E8005420700280F8758F0275A700D2AF7598F2
:1008F8000075A90C75A70F75AB4375ADFB75AC1EDC
:1009080075A700758911758E00758C00758A00D2DF
:10091800A9D28C758D00758B00D2ABD28E75CD00A7
:1009280075CC0075CA0075CB00D2ADC2CFD2CA75DE
:1009380091047592007593CD75EF0675D94075CF02
:1009480001900786E4F0A3F0751300751400C299AE
:10095800D20D74C8F518751700122B2475A70FE56A
:10096800FB90001AF0E5FA90001BF0E5F990001CE6
:10097800F075A70090F800E493F508122C5B12318B
:1009880095900789E0900026F090078AE09000276C
:10099800F090078BE0900028F090078CE0900029F9
:1009A800F090078DE0F56690078EE0F56890078F68
:1009B800E0F569900790E0F56A900791E0F5659099
:1009C8000792E0F567900793E0F564900794E0F5E7
:1009D80063900795E090002AF0900796E090002B2E
:1009E800F0900797E090002CF0900798E090004175
:1009F800F0900799E0900042F090079AE090004349
:100A0800F090079BE0900044F090079CE090004530
:100A1800F090079DE0900046F090079EE090004718
:100A2800F090079FE0900048F09007A0E090003316
:100A3800F09007A1E0900034F09007A2E090003514
:100A4800F09007A3E0900036F07400900082F090D8
:100A5800013AE0700C90013BE0700690013CE060C8
:100A6800028004C20D8002D20D90F807E493900032
:100A780021F0900021E0440A900021F0900021E04C
:100A880054FE900021F07406900012F07402900059
:100A980013F090F802E493900014F074039000159A
:100AA800F07403900016F07402900017F07405902B
:100AB8000018F0900014E0B404067404900018F0D4
:100AC800900014E0B403067403900018F0740490C6
:100AD8000019F090F804E49390001DF07400900061
:100AE8001EF090F805E49390001FF090F806E49348
:100AF800900020F074FF900022F0744C900125F0D3
:100B08007465900126F07478900127F0747590014F
:100B180028F07473900129F0742090012AF0744130
:100B280090012BF0743690012CF0743590012DF063
:100B3800743090012EF0744590012FF074209001CC
:100B480030F07435900131F07453900132F07450E4
:100B5800900133F090007AE0D3940140067400903D
:100B6800007AF0755801755901740390004CF01221
:100B780000C91204E5900014E0B40405120671805F
:100B880011900014E0D3940440051205A3800312C9
:100B9800073F122B50E5B554FEF5B5900025E4F05B
:100BA800900786E4F0A3F0752400752300754800CB
:100BB800752A007529007549007532007531007570
:100BC8004A00755400755500755A007551057552DF
:100BD8000175343C7533007571007570007572CD00
:100BE80075560075570075430075440075450075C6
:100BF8004600755B0075470075420075410090001E
:100C080006E4F0A3F0900008E4F0A3F0755E007528
:100C18005F0090000E74FDF0A374E8F0900023E4E8
:100C2800F07464900024F0C200D201C202D203C260
:100C380009756D00C20A754D00756E00C2A1C2A289
:100C4800C287C290E5B554BFF5B5C20F7E017F00DB
:100C5800900028E01243F1900027E02FFF50010E8A
:100C680090000AEEF0A3EFF0900026E0700674FF03
:100C7800900026F090000AE0FEA3E0FFEFD394FF77
:100C8800EE940F400790000AE4F0A3F0740090007F
:100C980071F07400900079F07400900082F0740094
:100CA80090008DF074009000B4F0E56770037567EC
:100CB80004743A90074EF074FD90074FF0900414B6
:100CC800E0900454F0D2B0D2B7D2A7D2A6D2B1D213
:100CD800A3C207C208A2B6B39204A2B3B39205D2C4
:100CE8009CD2EC75CF01A298B34005C2981234F992
:100CF800E5136006A299B3B340028005C299123A7F
:100D08006FE51464016005E514B4040280D5E54D6F
:100D1800D39405400CE55AC394C85002055A754D42
:100D280000E572C394F0501A787012003FAE70AFAD
:100D380071EFD394E8EE940340080572757100755D
:100D48007000C28E7E047F00E54C1243F1E58D757C
:100D5800F004A4FDACF0EF2DFDEE3CFCE58B75F046
:100D68004084FF7E00ED2FFFEC3EFE8E258F26D2BD
:100D78008EA2B6300401B35003020EB9A2B63004F5
:100D880001B35003020EB9A2B6405A0554E5B54462
:100D980001F5B5900024E4F0E554D3956640447C11
:100DA800817D991241FB8E238F24E5482FFF500146
:100DB8000E74011243E38E238F2485244875540151
:100DC800C28E758D00758B00754C00D28E7403BE73
:100DD80000039F50069000257401F0E543B4060314
:100DE800754300D204A2B6B35003020EB9C20490F0
:100DF800006BE06018123BB0A200B34008E5B544B0
:100E080008F5B58006E5B554F7F5B58002C200903F
:100E1800006EE06018123D05A202B34008E5B54433
:100E280002F5B58006E5B554FDF5B58006E5B5547F
:100E3800FDF5B5A207B34004D2878002C2879000AF
:100E480059E06004D2908002C29090004AE0B40158
:100E580004D2A18002C2A1900049E0B40104D2A248
:100E68008002C2A2A20CB34008E5B54440F5B580A3
:100E780006E5B554BFF5B5900018E0FE900014E003
:100E8800C39E4009900014E0D39408400974FB9075
:100E98000023F01204AB90001DE0601590001DE0E7
:100EA800FE900017E06E600974FE900023F01204B3
:100EB800ABC2CA7E017F00E54E1243F1E5CD2FFF9C
:100EC80050010E8E278F28D2CAE565B401489000DC
:100ED8000EE0FCA3E0FDEFC39DEE9C4039B20BE5AC
:100EE8002A45296013A20BB34008E5B54404F5B5BB
:100EF8008006E5B554FBF5B590000EE0FEA3E0FFD3
:100F0800900010E0FCA3E0FDEF2DFDEE3CFC90000E
:100F18000EECF0A3EDF0A2B3300501B35003020FBD
:100F2800FEA2B3300501B35003020FFEA2B3500373
:100F3800020FF70555E5B54401F5B5900024E4F036
:100F4800E555D395685003020FF57CEA7D60AE271E
:100F5800AF281241FB8E298F2AE5691243F174FFED
:100F68008E048F05FF1243D38C298D2AE5492DFD68
:100F780050010C74018C068D071243E38E298F2AC9
:100F8800852A49A20CB3401574641243F190006796
:100F9800E08E048F05FF1243D38C298D2A755501E5
:100FA80090000EE0FEA3E0FFAC27AD2812000390EE
:100FB800000EEEF0A3EFF0E567FF1243D3740AFFCB
:100FC8001243D390007BE08C068D071243F1741412
:100FD8008E048F05FF1243D3900010ECF0A3EDF0C0
:100FE800C2CA75CD0075CC00754E00D2CAD205A212
:100FF800B3B34002C205900025E0B40107E556C32B
:1010080094064003021B79E56E902AF1F8282873AC
:10101800900059E0C39402400302116CE551D39447
:1010280001500302116CE55175F040A4FFAEF09039
:10103800031212001EE0C395455018E55175F040A3
:10104800A4FFAEF090031112001EE0F52E752D00DE
:1010580002116CE55175F040A4FFAEF09003101238
:10106800001EE0C395454003021108E55175F040A4
:10107800A4FFAEF090031112001EE55175F040A4D4
:10108800FFAEF0E0FC90030F12001EECFEE0FFEE56
:10109800C39FFEE5518E0475F040A4FFAEF09003A7
:1010A8001012001EE0F40425458C0088F0A4FFAE61
:1010B800F0E5518F048E0575F040A4FFAEF0900363
:1010C8001212001EE55175F040A4FFAEF0E0FA9050
:1010D800031012001EEAFEE0FFEEC39FFECDCCCD4A
:1010E8008E071243D3E55175F040A4FFAEF090038C
:1010F8000F12001EE02DFD50010C8C2D8D2E8064EA
:10110800E55175F040A4FFAEF090030F12001EE504
:101118005175F040A4FFAEF0E0FC90030E12001EE3
:10112800ECFEE0FFEEC39F8545F0A4FFAEF0E5516D
:101138008F048E0575F040A4FFAEF09003101200E6
:101148001EE0FECDCCCD8E071243D3E55175F0409D
:10115800A4FFAEF090030E12001EE02DFD50010C0E
:101168008C2D8D2E756E01021B79900059E0C39469
:101178000240030212C890004FE0D3955150030279
:1011880012C8E55175F040A4FFAEF09003181200A4
:101198001EE0C395455018E55175F040A4FFAEF028
:1011A80090031712001EE0F52C752B000212C8E5FB
:1011B8005175F040A4FFAEF090031612001EE0C374
:1011C80095454003021264E55175F040A4FFAEF066
:1011D80090031712001EE55175F040A4FFAEF0E031
:1011E800FC90031512001EECFEE0FFEEC39FFEE527
:1011F800518E0475F040A4FFAEF090031612001E45
:10120800E0F40425458C0088F0A4FFAEF0E5518F8A
:10121800048E0575F040A4FFAEF090031812001E6E
:10122800E55175F040A4FFAEF0E0FA900316120005
:101238001EEAFEE0FFEEC39FFECDCCCD8E07124323
:10124800D3E55175F040A4FFAEF090031512001ECF
:10125800E02DFD50010C8C2B8D2C8064E55175F030
:1012680040A4FFAEF090031512001EE55175F04042
:10127800A4FFAEF0E0FC90031412001EECFEE0FFA9
:10128800EEC39F8545F0A4FFAEF0E5518F048E05AF
:1012980075F040A4FFAEF090031612001EE0FECDDC
:1012A800CCCD8E071243D3E55175F040A4FFAEF0C4
:1012B80090031412001EE02DFD50010C8C2B8D2C78
:1012C800756E02021B79900059E0B4022AE5517547
:1012D800F040A4FFAEF090031712001EE0F52C7545
:1012E8002B00E55175F040A4FFAEF090030E1200FC
:1012F8001EE0F52E752D00900059E0B4030F900004
:1013080051E0F52C752B00752E00752D00E551B4B4
:101318000105756E048017E551B40205756E0580E8
:101328000DE551B40305756E068003756E03021B47
:1013380079E551D394034015E55175F040A4FFAE0B
:10134800F090032012001EE0C3955A4002807DAE43
:1013580023AF24AC2DAD2EEDD39FEC9E401AE55162
:1013680075F040A4FFAEF090031E12001EE0A829FD
:10137800B80005D3952A500280021551E551B5529F
:1013880037E551C395605030E55604D39551402850
:10139800AE23AF24AC2BAD2CEFD39DEE9C4019E5CA
:1013A8005175F040A4FFAEF090031F12001EE0A894
:1013B80029B80006952A400280020551C292E551DB
:1013C80065526008C207755A00756DFA756E080295
:1013D8001B79E551B40115E55175F040A4FFAEF055
:1013E80090032012001EE0C3955A40028050A209C3
:1013F800B34011C209755102D20AD208756DCD7574
:101408005A008038E551C395605031AE23AF24AC03
:101418002BAD2CEFD39DEE9C400D90039FE0A829A7
:10142800B80006952A40028002D209A209B3400CEE
:10143800900360E0C39405F55A756DFAC292756E13
:1014480007021B79E551B40215E55175F040A4FF78
:10145800AEF090032012001EE0C3955A4003021418
:10146800F5900049E0701DAE23AF24AC2DAD2EEDF4
:10147800D39FEC9E400E90039EE0A829B80005D3A8
:10148800952A50028003755101A209B34009C20987
:10149800755103D2088041E551C39560503AAE2397
:1014A800AF24AC2BAD2CEFD39DEE9C4014E556D366
:1014B8009401400D9003DFE0A829B80006952A4062
:1014C800028002D209A209B3400E9003A0E0C3949F
:1014D80002F55A756DFAD208E5516552600D755AD4
:1014E80000E551B40105C208756DFAC292756E0720
:1014F800021B79E551B40315E55175F040A4FFAE20
:10150800F090032012001EE0C3955A400302159C78
:10151800A209B3400EC209755102D20AD208756DEC
:10152800CD802DAE23AF24AC2DAD2EEDD39FEC9EF8
:10153800400E9003DEE0A829B80005D3952A500292
:10154800800ED2099003E0E0C39405F55A756DFA50
:10155800E551C395605023E556D39402401CAE2351
:10156800AF24AC2BAD2CEFD39DEE9C400D90042006
:10157800E0A829B80006952A40028003755104E5C1
:10158800516552600DE551B40405C207756DFA75D1
:101598005A00C292756E07021B79E55175F040A496
:1015A800FFAEF090031A12001EE0B40117E5517562
:1015B800F040A4FFAEF090032012001EE0241EC3EA
:1015C800955A4003021672753064752F00A207B34E
:1015D800500B900060E02405C39545400302167245
:1015E800E55175F040A4FFAEF090031D12001EE017
:1015F800C395454064E55175F040A4FFAEF09003F3
:101608001C12001EE55175F040A4FFAEF0E0FC90FE
:10161800031B12001EECFEE0FFEEC39F8545F0A4FD
:10162800FFAEF0E5518F048E0575F040A4FFAEF0D3
:1016380090031D12001EE0FECDCCCD8E071243D3C1
:10164800E55175F040A4FFAEF090031B12001EE0B8
:101658002DFD50010C8C2F8D30AE23AF24AC2FAD57
:1016680030EFD39DEE9C4002D207756E09021B79BC
:10167800E55175F040A4FFAEF090031A12001EE089
:10168800B40117E55175F040A4FFAEF090032012A5
:10169800001EE0240AC3955A4003021748753064B7
:1016A800752F00A207B3500B900060E02405C39586
:1016B800454003021748E55175F040A4FFAEF0908D
:1016C800031D12001EE0C395454064E55175F040C6
:1016D800A4FFAEF090031C12001EE55175F040A463
:1016E800FFAEF0E0FC90031B12001EECFEE0FFEEE4
:1016F800C39F8545F0A4FFAEF0E5518F048E0575B4
:10170800F040A4FFAEF090031D12001EE0FECDCC09
:10171800CD8E071243D3E55175F040A4FFAEF0908B
:10172800031B12001EE02DFD50010C8C2F8D30AED6
:1017380023AF24AC2FAD30EFD39DEE9C4002D207EF
:10174800756E09021B79E55AB41603756DCDE5511E
:10175800B40205A209B3400302186DE55AC3940AFE
:10176800507D900072E0B40258E54575F00284FFA0
:101778007E0090018012001EE0F572E54775F00AC0
:1017880084FF7E0090024E12001EE0F55DE5722592
:101798005DD39464400BE572255DC39464F5728053
:1017A80003757200E57275F00284FF7E008F72EF98
:1017B800C394335007EF24CDF57280037572FF8010
:1017C8001CE54575F00284FF7E0090018012001E22
:1017D800E075F00284FF7E00EF24CDF572807B90E7
:1017E8000072E0B40258E54575F00284FF7E00906F
:1017F80001B212001EE0F572E54775F00A84FF7E1B
:101808000090024E12001EE0F55DE572255DD3944E
:1018180064400BE572255DC39464F57280037572AC
:1018280000E57275F00284FF7E008F72EFC3943377
:101838005007EF24CDF57280037572FF801CE545D3
:1018480075F00284FF7E009001B212001EE075F070
:101858000284FF7E00EF24CDF572E55AD39402404E
:1018680004C2A0C20AE551B40206A209B3B34002F9
:10187800807B900072E0B40258E54575F00284FF61
:101888007E009001B212001EE0F572E54775F00A7D
:1018980084FF7E0090024E12001EE0F55DE5722581
:1018A8005DD39464400BE572255DC39464F5728042
:1018B80003757200E57275F00284FF7E008F72EF87
:1018C800C394335007EF24CDF57280037572FF80FF
:1018D8001CE54575F00284FF7E009001B212001EDF
:1018E800E075F00284FF7E00EF24CDF572E551B477
:1018F8000307E55AC394194003021986900072E061
:10190800B40258E54575F00284FF7E009001B212DA
:10191800001EE0F572E54775F00A84FF7E0090022C
:101928004E12001EE0F55DE572255DD39464400B10
:10193800E572255DC39464F5728003757200E572E3
:1019480075F00284FF7E008F72EFC394335007EF67
:1019580024CDF57280037572FF801CE54575F00291
:1019680084FF7E009001B212001EE075F00284FF31
:101978007E00EF24CDF572E55AB41602C208756EE2
:101988000A021B79E551D394034006E55A640A60BC
:10199800028003756DCDE55164026010900050E03F
:1019A8002402A823B80005D3952450028002C20758
:1019B800E551B40119A209B35014E545C394055083
:1019C8000D90035FE0A829B80006952A4002800E12
:1019D800D209900360E0C39405F55A756DFA90003A
:1019E80059E0C39403503BE551D394014034E55189
:1019F80075F040A4FFAEF090031412001EE0A82377
:101A0800B8001FD39524401AE55175F040A4FFAEE5
:101A1800F090031F12001EE0A829B80005D3952AEC
:101A280050028052E55164036015900049E070044B
:101A380015518009E551D3940340021551802AA21B
:101A480009B350099003E0E0C3955A4002801AE5B3
:101A580045C394055005755101800ED2099003E0E5
:101A6800E0C39405F55A756DFAE551B40108C2074B
:101A7800C208C2A0C209756E0B021B79E551D39446
:101A880001402FE55175F040A4FFAEF0900312120B
:101A9800001EE0C39545501AE55175F040A4FFAE0D
:101AA800F090031E12001EE0A829B80005D3952A5D
:101AB80050028033E551B40305A209B34002800EF9
:101AC800D2099003E0E0C39405F55A756DCDE55150
:101AD80064036013900049E0700415518009E551D2
:101AE800D3940340021551E551D394034021E556A0
:101AF800C39403501AE55175F040A4FFAEF090036B
:101B08001E12001EE0A829B80005D3952A500280AD
:101B180009E551D3940340021551E551B4031FE57B
:101B280056B4011AE55175F040A4FFAEF090031EBB
:101B380012001EE0A829B80005D3952A5002801A81
:101B4800E551B40305A209B34002800ED2099003FF
:101B5800E0E0C39405F55A756DCD900060E0D3952B
:101B6800455009900054E0C395455002C207756E70
:011B7800006C
:102AF1000210180211720212CE0213390213DA0205
:102B0100144C0214FB0215A202167802174E021988
:042B11008C021A8494
:101B7900900059E07003021DCEA2A5B34008A2A4AB
:101B8900B34003021DB7AE35AF367441D39F749C81
:101B99009E4005783512003FAE35AF36EFB4880662
:101BA900EEB413028003021D79A2A55003021CA8FA
:101BB900900059E0B4010B90004FE0D395604002CA
:101BC9000560900059E0B4027590004FE0D395513B
:101BD9004019E55175F040A4FFAEF09003141200CE
:101BE9001EE0A823B8000695244002804BE551B4B5
:101BF900010ED209900360E0C39405F55A756DFA98
:101C0900E551B40207E556D3940150028010D20978
:101C19009003A0E0C39405F55A756DFAD208E55111
:101C2900D394024007E556D394025002800A055125
:101C3900C207755A00756DFA90004FE0F560900083
:101C490059E0B4035A90004FE0D39551404BE55108
:101C5900B4010ED209900360E0C39405F55A756D7D
:101C6900FAE551B40207E556D3940150028013D224
:101C7900099003A0E0C39405F55A756DFAD2087569
:101C89005A00E551D394024007E556D39402500215
:101C990080070551C207756DFA90004FE0F560A203
:101CA900A45003021D79900059E0B40150E551D3C5
:101CB90094014046E55175F040A4FFAEF090031E33
:101CC90012001EE0A829B8002CD3952A4027E55117
:101CD900B40313D2099003E0E0C39405F55A756D76
:101CE900FA756002800D1551855160756DFA755A46
:101CF90000C2088003855160800375600190005916
:101D0900E0D39401405EE551D394014034E5517527
:101D1900F040A4FFAEF090031112001EE0A823B812
:101D2900001FD39524401AE55175F040A4FFAEF089
:101D390090031E12001EE0A829B80005D3952A5069
:101D4900028021E551B40310D2099003E0E0C39465
:101D590005F55A756DFA800C1551756DFA755A00AD
:101D6900C207C208E556B40704055E8003755E0024
:101D7900E563B4010EAE35AF36EF64407005EE642D
:101D89009C6002800EA2A54003755801A2A44003DD
:101D9900755802E563B4020EAE35AF36EF64407094
:101DA90005EE649C6002800690004FE0F560A2A5F4
:101DB900B3B35006A2A4B3B34002800675360075CA
:101DC9003500021ECFA2A5B34008A2A4B340030266
:101DD9001EBBAE35AF367441D39F749C9E400578C7
:101DE9003512003FAE35AF36EFB48806EEB41302B4
:101DF9008003021EBBA2A5406F900068E0605A9064
:101E0900004AE0B4010790004AE4F0800690004AD5
:101E19007401F090004AE0700575600480037560F4
:101E29000590004AE0B40104D2A18002C2A1E551A3
:101E3900B4051AE55175F040A4FFAEF090031E12E7
:101E4900001EE0A829B80005D3952A50028008751C
:101E59005104C207755A008003756005E556B40739
:101E690004055E8003755E00A2A44046900069E007
:101E79006034900049E0B40107900049E4F080061D
:101E89009000497401F0900049E0B40117D2A2E52D
:101E990051B4010ED209900360E0C39405F55A7557
:101EA9006DFA8002C2A2E556B40704055E80037587
:101EB9005E00A2A5B3B35006A2A4B3B34002800644
:101EC900753600753500E55865596006900082E061
:101ED9006003022057C29C751400751300C2CAE53D
:101EE90058902B15F82828738012123195800D12FD
:0C1EF900326E8008123347800312342040
:0F2B1500021EF1021EF3021EF8021EFD021F0235
:101F0500900029E090007AF0E566900057F0E568CA
:101F1500900062F0E569900063F0E56A900074F066
:101F2500E56590007CF0E56790007DF0E564900044
:101F350080F0E563900081F090002AE090013AF08E
:101F450090002BE090013BF090002CE090013CF0DC
:101F5500900041E0900090F0900042E0900091F0F8
:101F6500900043E0900092F0900044E0900093F0E0
:101F7500900045E0900094F0900046E0900095F0C8
:101F8500900047E0900096F0900048E0900097F0B0
:101F9500900033E0900099F0900034E090009AF0C2
:101FA500900035E090009BF0900036E090009CF0AA
:101FB5007400900082F0744C900125F074659001D6
:101FC50026F07478900127F07475900128F07473E9
:101FD500900129F0742090012AF0744190012BF0B2
:101FE500743690012CF0743590012DF07430900109
:101FF5002EF0744590012FF07420900130F0743567
:10200500900131F07453900132F07450900133F027
:10201500900414E0900454F0743A90074EF074FD67
:1020250090074FF01200C9900004E4F0A3F090006F
:10203500067475F0A37430F09000087475F0A374FD
:1020450030F0855859D2CA754C00D29C741B90004B
:1020550023F0E556C394065005E551B55203022019
:10206500EDC207E55175F040A4FFAEF090032212D2
:10207500001EE030E003D38001C39296E55175F070
:1020850040A4FFAEF090032312001EE030E003D31E
:102095008001C39295E55175F040A4FFAEF0900321
:1020A5002412001EE030E003D38001C392A0E55165
:1020B50075F040A4FFAEF090032512001EE030E05D
:1020C50003D38001C39297A20AB34002D2A08551DF
:1020D50052AE29AF2A7405BE00039F5007E545D3CC
:1020E500940550028002D292E556D394055003021E
:1020F500223AC207E551D39401500302218FE551DD
:1021050075F040A4FFAEF090031E12001EE0A82952
:10211500B80007D3952A40021551E551655260670D
:10212500E55175F040A4FFAEF090032212001EE0C9
:1021350030E003D38001C39296E55175F040A4FFCA
:10214500AEF090032312001EE030E003D38001C3FC
:102155009295E55175F040A4FFAEF090032412006E
:102165001EE030E003D38001C392A0E55175F04035
:10217500A4FFAEF090032512001EE030E003D380EB
:1021850001C3929785515202223AE556B40634901E
:1021950000ACE030E003D38001C392969000ADE03F
:1021A50030E003D38001C392959000AEE030E003A8
:1021B500D38001C392A09000AFE030E003D380014B
:1021C500C39297E556B407349000A5E030E003D3F9
:1021D5008001C392969000A6E030E003D38001C34E
:1021E50092959000A7E030E003D38001C392A090C0
:1021F50000A8E030E003D38001C39297E556B40808
:102205003490009EE030E003D38001C392969000A5
:102215009FE030E003D38001C392959000A0E030A9
:10222500E003D38001C392A09000A1E030E003D386
:102235008001C39297E54575F00284FF7E00900109
:102245004E12001EE075F00284FF7E00EF24CDF5EE
:102255005CE595C3955C4004C2938002D293A208C5
:10226500B34002800FA207B34007E556D39405405B
:10227500037572CDE595C395724004C2948002D270
:1022850094E595C3956D4004C2918002D291E543D2
:10229500C394064003022896A2EDB3500302289684
:1022A500C2EDE54360030223F87E017F00E5BE121F
:1022B50043F1E5BD2FFF50010E900000EEF0A3EFB6
:1022C500F0900029E0B401177E0F7FFF900000E039
:1022D500FCA3E0FD120003900000EEF0A3EFF090E8
:1022E5000079E0B4025B900000E0FEA3E0FF9000FF
:1022F5000AE0FCA3E0FDEDD39FEC9E400F900000AB
:10230500E0F8A3E090000AC8F0A3C8F0900000E050
:10231500FEA3E0FF90000CE0FCA3E0FDEFD39DEEF3
:102325009C400F900000E0F8A3E090000CC8F0A3DB
:10233500C8F0900000E0FEA3E0FF74041243E38FB1
:1023450044900079E07060900000E0FEA3E0FF900B
:10235500000AE0FCA3E0FDEFD39DEE9C400D1200CA
:1023650003900000EEF0A3EFF08007900000E4F08A
:10237500A3F0900000E0FEA3E0FF74101243F1907B
:102385000026E08E048F05FF1243D3900000ECF089
:10239500A3EDF07400D39D74019C4008900001E00A
:1023A500F54480037544FFE54475F00AA4FFAEF0DB
:1023B50074198E048F05FF1243D38D45ED2532FF29
:1023C500AE3150010E74011243E38F4585453275D8
:1023D5003100EFD394624003754562900072E0646A
:1023E500016006900066E060028005754301800388
:1023F50075BB17E543B4010280030224E87E017F23
:1024050000E5BE1243F1E5BD2FFF50010E9000001F
:10241500EEF0A3EFF0900072E0B4017EE5344533B1
:102425006025AC33AD341DBDFF011C8F028E038CBE
:10243500068D07903F2712002EE493FE740193FF4B
:10244500EFC39AEE9B40028005783312441BAE33EE
:10245500AF3474B3BE0025D39F4021900000E0FC4B
:10246500A3E0FD0FBF00010E903F2712002EE4935D
:10247500FE740193FFEDC39FEC9E40028005783307
:1024850012003FAE33AF34E56A1243F174648E0433
:102495008F05FF1243D38D478033900066E0602D92
:1024A500900000E0FEA3E0FFEFD39400EE94084017
:1024B5000F900066E0B40104C20C8002D20C800DBE
:1024C500900066E0B40104D20C8002C20C90007248
:1024D500E064026006900066E0600575BB16800347
:1024E500754302E543B4020280030225D67E017FCF
:1024F50000E5BE1243F1E5BD2FFF50010E9000002F
:10250500EEF0A3EFF0900072E0B4027EE5344533BF
:102515006025AC33AD341DBDFF011C8F028E038CCD
:10252500068D0790409112002EE493FE740193FFEF
:10253500EFC39AEE9B40028005783312441BAE33FD
:10254500AF3474B3BE0025D39F4021900000E0FC5A
:10255500A3E0FD0FBF00010E90409112002EE49301
:10256500FE740193FFEDC39FEC9E40028005783316
:1025750012003FAE33AF34E56A1243F174648E0442
:102585008F05FF1243D38D478033900066E0602DA1
:10259500900000E0FEA3E0FFEFD39400EE94084026
:1025A5000F900066E0B40104C20C8002D20C800DCD
:1025B500900066E0B40104D20C8002C20C90007257
:1025C500E07003754700900066E07002C20C75BBB1
:1025D5001FE543B403457E017F00E5BE1243F1E5E7
:1025E500BD2FFF50010E900000EEF0A3EFF074092F
:1025F5001243F174E68E048F05FF1243D38C418D8F
:1026050042E54A2DFD50010C74018C068D071243DD
:10261500E38E418F4285424A75BB19E543B40402F6
:10262500800302277E7E017F00E5BE1243F1E5BDF2
:102635002FFF50010E900000EEF0A3EFF07404128E
:1026450043E38F4BE564B40102800302270B756BEE
:1026550000756B00E56BD3940740030226F8E56B24
:10266500900041124409E0D3954B501AE56B900058
:1026750041124409E0F404254BFEE56B9000371246
:102685004409EEF08017E56B900041124409E0C360
:10269500954BFEE56B900037124409EEF0E56BC3F0
:1026A50094044009900084E0C3956B503BE56B6052
:1026B50029E56B900037124409FEE0FFEE90003FDC
:1026C500E0D39F4013E56B900037124409E090007A
:1026D5003FF0E56B900040F0800E900037E09000F1
:1026E5003FF07400900040F0786B740126F64003CB
:1026F500022659900040E0F4042408F556E556D327
:1027050094054002C292E564D39401402FE54BD372
:10271500946E4004D2108002C210755605E564B46B
:102725000205A210B340028003755607E564B403A1
:1027350006A210B3B340028003755607E5576556E8
:102745006008E55104F552855657E556B40708E586
:10275500B54480F5B58006E5B5547FF5B5E5566415
:10276500066005E556B40808E5B54410F5B58006DC
:10277500E5B554EFF5B575BB13E543B40502800324
:102785000228927E017F00E5BE1243F1E5BD2FFFD1
:1027950050010E900000EEF0A3EFF074041243E335
:1027A5008F46E563B40202800302288F756B0075BE
:1027B5006B00E56BD394034003022846E56B90005C
:1027C50033124409E0D39546501AE56B9000331255
:1027D5004409E0F4042546FEE56B90002D124409FA
:1027E500EEF08017E56B900033124409E0C395467F
:1027F500FEE56B90002D124409EEF0E56B6029E5CE
:102805006B90002D124409FEE0FFEE900031E0D3FD
:102815009F4013E56B90002D124409E0900031F0C4
:10282500E56B900032F0800E90002DE0900031F0C5
:102835007400900032F0786B740126F6400302278D
:10284500B7900082E07043E52A45296036E558C314
:102855009403500A900032E004C3940340028007B9
:10286500900032E004F558E558D39402400A9000F0
:1028750032E004D3940250028007900032E004F560
:10288500588007900032E004F55875BB180543D20F
:10289500ECE55ED3940450030229C275CF01C293BF
:1028A500AE35AF367488D39F74139E4005A2A5B389
:1028B5004014AE35AF367488D39F74139E4005A27D
:1028C500A4B340028058783512003FAE35AF36EFDD
:1028D500B4884BEEB41347A2A5B3500990004FE05E
:1028E500D395515002800C0551E551B40203755141
:1028F500038011A2A5B3500890004FE06551600216
:102905008002D207A2A4B35007E551D39401500227
:10291500800C1551E551B40203755101C207A2A5FA
:10292500B3B35006A2A4B3B3400280067536007552
:102935003500E55165526069E55175F040A4FFAE7B
:10294500F090032212001EE030E003D38001C39211
:1029550096E55175F040A4FFAEF090032312001EDA
:10296500E030E003D38001C39295E55175F040A4B2
:10297500FFAEF090032412001EE030E003D3800187
:10298500C392A0E55175F040A4FFAEF09003251267
:10299500001EE030E003D38001C39297C2948551B5
:1029A50052A20740057572CD80037572FFE595C388
:1029B50095724004C2948002D2940228A0AE25AF3D
:1029C50026EFD39420EE944E5003022AC51204AB91
:1029D500C28E758D00758B00754C00D28EC2077541
:1029E50071007570007572CD7551057524007523DC
:1029F50000755400755A00C287900059E06004D2F2
:102A0500908002C29090004AE0B40104D2A18002F5
:102A1500C2A1900049E0B40104D2A28002C2A2A2E0
:102A25000CB34008E5B54440F5B58006E5B554BF9F
:102A3500F5B590006BE06018123BB0A200B34008FA
:102A4500E5B54408F5B58006E5B554F7F5B580025A
:102A5500C20090006EE06018123D05A202B3400866
:102A6500E5B54402F5B58006E5B554FDF5B5800636
:102A7500E5B554FDF5B590000E74FDF0A374E8F0CE
:102A8500E543B40603754300900025E4F075260080
:102A9500752500758D00758B00754C00900024E040
:102AA500C394035008900024E004F080067403905A
:102AB5000024F0900024E0B40306E5B554FEF5B516
:102AC500AE27AF28EFD39410EE9427401CC2CA75E9
:102AD500CD0075CC00752800752700D2CA754E004B
:0C2AE500752A00752900755500020CEBE5
:103EB700000001000132016401960196020002121E
:103EC70002240200020003000340038003C0040031
:103ED7000440048004C00500060006000600060032
:103EE700060006000600060000FF01310163019588
:103EF70001FF01FF0211022302FF02FF02FF033F3E
:103F0700037F03BF03FF043F047F04BF04FF05FFD4
:103F170006FF06FF06FF06FF06FF06FF06FF06FF72
:103F27000FAA0FA50F9F0F9A0F940F8D0F870F8062
:103F37000F780F710F680F600F570F4E0F450F3B2C
:103F47000F300F250F1A0F0E0F020EF50EE80EDBBE
:103F57000ECC0EBE0EAE0E9F0E8E0E7D0E6C0E5A42
:103F67000E470E340E200E0C0DF70DE20DCB0DB5DE
:103F77000D9D0D850D6D0D540D3A0D200D050CE9A8
:103F87000CCE0CB10C940C760C580C3A0C1B0BFB9A
:103F97000BDB0BBB0B9A0B790B570B350B130AF18A
:103FA7000ACE0AAB0A870A640A400A1C09F809D430
:103FB70009B0098C09670943091F08FB08D608B22D
:103FC700088E086A0846082307FF07DC07B9079623
:103FD70007730751072F070D06EC06CA06AA0689BD
:103FE70006690649062A060A05EC05CD05B00592BD
:103FF70005750558053C0520050504EA04CF04B5F9
:10400700049C04820469045104390422040B03F458
:1040170003DE03C803B2039D038903750361034DE0
:10402700033B03280316030402F202E102D102C094
:1040370002B002A00291028202730265025702498E
:10404700023C022F02220216020901FD01F201E6DB
:1040570001DB01D001C601BB01B101A7019D01949C
:10406700018B0182017901700168016001580150DB
:104077000148014101390132012B0125011E0118B7
:104087000111010B010500FF00FA0FA60FA00F9900
:104097000F920F8B0F840F7C0F740F6B0F620F58EB
:1040A7000F4E0F430F380F2C0F1F0F120F050EF770
:1040B7000EE80ED80EC80EB70EA50E930E800E6C26
:1040C7000E580E420E2C0E150DFD0DE40DCB0DB145
:1040D7000D950D790D5D0D3F0D200D010CE10CC007
:1040E7000C9E0C7C0C590C350C100BEA0BC40B9E68
:1040F7000B760B4F0B260AFD0AD40AAA0A800A552B
:104107000A2A09FF09D409A8097C0950092508F9D1
:1041170008CD08A10875084A081E07F307C8079DB8
:1041270007730749072006F706CE06A6067E065739
:104137000630060A05E405BF059B057705540532D9
:10414700051004EF04CE04AE048F04710453043544
:10415700041903FD03E203C703AD0394037B036361
:10416700034B0334031E030802F302DE02CA02B63E
:1041770002A30291027F026D025C024C023C022CF8
:10418700021D020E020001F201E401D701CA01BEBD
:1041970001B101A6019A018F0185017A01700166BB
:1041A700015D0153014A0141013901310129012111
:1041B70001190112010B010400FD00F700F000EAEC
:1041C70000E400DE00D900D300CE00C900C400BF60
:1041D70000BA00B500B100AD00A800A400A0009C83
:1041E700009900950091008E008A00870084008165
:0441F700007E007BCB
:102B2400751A00751900AE19AF1AAC17AD18EDC3BC
:102B34009FEC9E401674FF1243C375CF01781A743C
:102B44000126F6500418E436F650DB22900786E49A
:102B5400F0A3F0751000750F00751300751400C212
:102B640011D21222C2AF75D900758F0375B7A5753E
:102B7400B7F190F800E4F0758F0175B7A575B7F15A
:102B8400E50890F800F075B7A575B7F190F801E481
:102B9400F075B7A575B7F190079DE090F802F07550
:102BA400B7A575B7F19007A1E090F803F075B7A544
:102BB40075B7F190079EE090F804F075B7A575B766
:102BC400F190079FE090F805F075B7A575B7F190FF
:102BD40007A0E090F806F075B7A575B7F19007A2C5
:102BE400E090F807F0758F0075D940D2AF229007B6
:102BF40088E0B4AB61C2AF75D90075B62275F52211
:102C0400758F0375B7A575B7F1740090F600F0756C
:102C14008F01750A00750900AE09AF0A7413BE006E
:102C2400279F402475B7A575B7F190078912001E38
:102C3400E0FC90F60012001EECF0780A740126F60F
:102C4400500418E436F650D0758F0075F51175B63A
:102C54002075D940D2AF22C2AF75D90075F522755F
:102C64000A00750900AE09AF0A7413BE00229F4022
:102C74001F90F60012001EE493FC90078912001EB8
:102C8400ECF0780A740126F6500418E436F650D5B0
:102C940075F51175D940D2AF22900788E0B4AA0225
:102CA4008003022DDAC2AF75D90075B62275F522FC
:102CB400758F0375B7A575B7F1740090EE00F075C4
:102CC400B7A575B7F1740090F000F075B7A575B7A6
:102CD400F1740090F200F075B7A575B7F174009027
:102CE400F400F0758F01750A00750900AE09AF0A8A
:102CF40074FFC39F74019E402475B7A575B7F19006
:102D0400004E12001EE0FC90EE0012001EECF07863
:102D14000A740126F6500418E436F650CF750A00FA
:102D2400750900AE09AF0A74FFC39F74019E402465
:102D340075B7A575B7F190024E12001EE0FC90F035
:102D44000012001EECF0780A740126F6500418E410
:102D540036F650CF750A00750900AE09AF0A74FF44
:102D6400C39F74019E402475B7A575B7F190044EB6
:102D740012001EE0FC90F20012001EECF0780A74BF
:102D84000126F6500418E436F650CF750A0075098A
:102D940000AE09AF0A74FFC39F74019E402475B747
:102DA400A575B7F190064E12001EE0FC90F40012D7
:102DB400001EECF0780A740126F6500418E436F686
:102DC40050CF758F0075F51175B62075D940D2AF07
:102DD400743A90074EF022900788E0B4AA02800368
:102DE400022F18C2AF75D90075B62275F522758FFA
:102DF4000375B7A575B7F1740090E600F075B7A533
:102E040075B7F1740090E800F075B7A575B7F17463
:102E14000090EA00F075B7A575B7F1740090EC0066
:102E2400F0758F01750A00750900AE09AF0A74FFC9
:102E3400C39F74019E402475B7A575B7F190004EE9
:102E440012001EE0FC90E60012001EECF0780A74FA
:102E54000126F6500418E436F650CF750A007509B9
:102E640000AE09AF0A74FFC39F74019E402475B776
:102E7400A575B7F190024E12001EE0FC90E8001216
:102E8400001EECF0780A740126F6500418E436F6B5
:102E940050CF750A00750900AE09AF0A74FFC39FCD
:102EA40074019E402475B7A575B7F190044E1200C5
:102EB4001EE0FC90EA0012001EECF0780A74012671
:102EC400F6500418E436F650CF750A00750900AEC2
:102ED40009AF0A74FFC39F74019E402475B7A5759A
:102EE400B7F190064E12001EE0FC90EC0012001E9A
:102EF400ECF0780A740126F6500418E436F650CF44
:102F0400758F0075F51175B62075D940D2AF743A36
:102F140090074EF022900788E0B4AA0280030230A2
:102F240056C2AF75D90075B62275F522758F037533
:102F3400B7A575B7F1740090DE00F075B7A575B745
:102F4400F1740090E000F075B7A575B7F1740090C6
:102F5400E200F075B7A575B7F1740090E400F07560
:102F64008F01750A00750900AE09AF0A74FFC39F8B
:102F740074019E402475B7A575B7F190004E1200F8
:102F84001EE0FC90DE0012001EECF0780A740126AC
:102F9400F6500418E436F650CF750A00750900AEF1
:102FA40009AF0A74FFC39F74019E402475B7A575C9
:102FB400B7F190024E12001EE0FC90E00012001ED9
:102FC400ECF0780A740126F6500418E436F650CF73
:102FD400750A00750900AE09AF0A74FFC39F740136
:102FE4009E402475B7A575B7F190044E12001EE0FB
:102FF400FC90E20012001EECF0780A740126F650F0
:103004000418E436F650CF750A00750900AE09AF0E
:103014000A74FFC39F74019E402475B7A575B7F168
:1030240090064E12001EE0FC90E40012001EECF02C
:10303400780A740126F6500418E436F650CF758FDA
:103044000075F51175B62075D940D2AF743A900762
:103054004EF022900788E0B4AA028003023194C2A1
:10306400AF75D90075B62275F522758F0375B7A5AE
:1030740075B7F1740090D600F075B7A575B7F17403
:103084000090D800F075B7A575B7F1740090DA0018
:10309400F075B7A575B7F1740090DC00F0758F0179
:1030A400750A00750900AE09AF0A74FFC39F740165
:1030B4009E402475B7A575B7F190004E12001EE02E
:1030C400FC90D60012001EECF0780A740126F6502B
:1030D4000418E436F650CF750A00750900AE09AF3E
:1030E4000A74FFC39F74019E402475B7A575B7F198
:1030F40090024E12001EE0FC90D80012001EECF06C
:10310400780A740126F6500418E436F650CF750A8E
:1031140000750900AE09AF0A74FFC39F74019E4095
:103124002475B7A575B7F190044E12001EE0FC900B
:10313400DA0012001EECF0780A740126F650041826
:10314400E436F650CF750A00750900AE09AF0A746B
:10315400FFC39F74019E402475B7A575B7F190060F
:103164004E12001EE0FC90DC0012001EECF0780A07
:10317400740126F6500418E436F650CF758F0075A6
:10318400F51175B62075D940D2AF743A90074EF058
:1031940022C2AF75D90075F522750A00750900AE13
:1031A40009AF0A74FFC39F74019E401F90EE001282
:1031B400001EE493FC90004E12001EECF0780A749A
:1031C4000126F6500418E436F650D4750A00750941
:1031D40000AE09AF0A74FFC39F74019E401F90F0B4
:1031E4000012001EE493FC90024E12001EECF078D4
:1031F4000A740126F6500418E436F650D4750A0011
:10320400750900AE09AF0A74FFC39F74019E401F85
:1032140090F20012001EE493FC90044E12001EEC87
:10322400F0780A740126F6500418E436F650D47582
:103234000A00750900AE09AF0A74FFC39F74019EAA
:10324400401F90F40012001EE493FC90064E1200FE
:103254001EECF0780A740126F6500418E436F65091
:10326400D475F51175D940D2AF22C2AF75D90075A6
:10327400F522750A00750900AE09AF0A74FFC39FF1
:1032840074019E401F90E60012001EE493FC90001F
:103294004E12001EECF0780A740126F6500418E46D
:1032A40036F650D4750A00750900AE09AF0A74FFEA
:1032B400C39F74019E401F90E80012001EE493FC1B
:1032C40090024E12001EECF0780A740126F65004A7
:1032D40018E436F650D4750A00750900AE09AF0A31
:1032E40074FFC39F74019E401F90EA0012001EE405
:1032F40093FC90044E12001EECF0780A740126F63A
:10330400500418E436F650D4750A00750900AE0965
:10331400AF0A74FFC39F74019E401F90EC0012001B
:103324001EE493FC90064E12001EECF0780A740121
:1033340026F6500418E436F650D475F51175D940C4
:10334400D2AF22C2AF75D90075F522750A0075098E
:1033540000AE09AF0A74FFC39F74019E401F90DE44
:103364000012001EE493FC90004E12001EECF07854
:103374000A740126F6500418E436F650D4750A008F
:10338400750900AE09AF0A74FFC39F74019E401F04
:1033940090E00012001EE493FC90024E12001EEC1A
:1033A400F0780A740126F6500418E436F650D47501
:1033B4000A00750900AE09AF0A74FFC39F74019E29
:1033C400401F90E20012001EE493FC90044E120091
:1033D4001EECF0780A740126F6500418E436F65010
:1033E400D4750A00750900AE09AF0A74FFC39F744F
:1033F400019E401F90E40012001EE493FC90064ED0
:1034040012001EECF0780A740126F6500418E43613
:10341400F650D475F51175D940D2AF22C2AF75D923
:103424000075F522750A00750900AE09AF0A74FF2C
:10343400C39F74019E401F90D60012001EE493FCAB
:1034440090004E12001EECF0780A740126F6500427
:1034540018E436F650D4750A00750900AE09AF0AAF
:1034640074FFC39F74019E401F90D80012001EE495
:1034740093FC90024E12001EECF0780A740126F6BA
:10348400500418E436F650D4750A00750900AE09E4
:10349400AF0A74FFC39F74019E401F90DA001200AC
:1034A4001EE493FC90044E12001EECF0780A7401A2
:1034B40026F6500418E436F650D4750A007509004F
:1034C400AE09AF0A74FFC39F74019E401F90DC00D5
:1034D40012001EE493FC90064E12001EECF0780AD3
:1034E400740126F6500418E436F650D475F51175B7
:1034F400D940D2AF22E51464046006E59964FF6004
:10350400028031A2114004D2118027E514600874AE
:10351400E62514900023F0E513600874F025139059
:103524000023F0E514B4010280FE75140075130045
:10353400C2118002C211E514903E5AF8282873750E
:103544001400E599B4FF03751301E599B4FE0375FE
:103554001302E599B4FD03751303E599B4FC0375EF
:103564001304E599B4FA03751305E599B4FB0675DC
:1035740014011204ABE599B4F9067514041204ABF2
:10358400E599D394E54007E599C394F04002801689
:103594008599157514027E017F00E515C394E61222
:1035A40043F18E0D8F0E900786E4F0A3F0E599D3D6
:1035B40094C44007E599C394E64002802885991590
:1035C40075140374E5C39515F50E750D00AE0DAFB6
:1035D4000E903EB712002EE493F874019390078680
:1035E400C8F0A3C8F0D299023A6E900786E0FEA311
:1035F400E0FFEFC39400EE94054009EFD394FFEE8F
:1036040094064013900786E0FEA3E0FF90004E125C
:10361400001EE599F0800385996C90078612000ED0
:10362400900786E0FEA3E0FFEFB40106EEB40702C4
:10363400800302387B90074EE0B43C0280030238DA
:103644007B75FFA0A20DB35005A20EB34003023751
:103654006EC29C90007AE090078CF0900057E09046
:10366400078DF0900062E090078EF0900063E09088
:10367400078FF0900074E0900790F090007CE09049
:103684000791F090007DE0900792F0900080E09028
:103694000793F0900081E0900794F090013AE09055
:1036A4000795F090013BE0900796F090013CE09084
:1036B4000797F0900090E0900798F0900091E090C8
:1036C4000799F0900092E090079AF0900093E090B0
:1036D400079BF0900094E090079CF0900095E09098
:1036E400079DF0900096E090079EF0900097E09080
:1036F400079FF0900099E09007A0F090009AE09066
:1037040007A1F090009BE09007A2F090009CE0904D
:1037140007A3F07400900082F01200C974AB900704
:0D37240088F0122BF274AA900788F0E55887
:063E5A000235430235EEC3
:10373100903E7BF82828738012122C9D800D122D4B
:0B374100DB8008122F198003123057A4
:0F3E7B0002373802373A02373F023744023749DD
:10374C00900788E4F090013AE0700C90013BE07037
:10375C000690013CE060028004C20D8002D20D0292
:10376C003870C29C900078E0900789F090005EE081
:10377C0090078AF090005FE090078BF090007AE061
:10378C0090078CF0900057E090078DF0900062E06D
:10379C0090078EF0900063E090078FF0900074E03B
:1037AC00900790F090007CE0900791F090007DE005
:1037BC00900792F0900080E0900793F0900081E0E9
:1037CC00900794F090013AE0900795F090013BE05F
:1037DC00900796F090013CE0900797F0900090E0F5
:1037EC00900798F0900091E0900799F0900092E08B
:1037FC0090079AF0900093E090079BF0900094E073
:10380C0090079CF0900095E090079DF0900096E05A
:10381C0090079EF0900097E090079FF0900099E041
:10382C009007A0F090009AE09007A1F090009BE028
:10383C009007A2F090009CE09007A3F07400900019
:10384C0082F074AB900788F0122BF274AA90078860
:10385C00F0122C9D122DDB122F19123057D29C75A1
:10386C0099FB80FED29C7514007513007599FB02B0
:10387C003A6E900786E0FEA3E0FFEF4E7006859946
:10388C0010750F00900786E0FEA3E0FF74016F4EE9
:10389C00701BAC0FAD10AA0DAB0EED2BFBEC3AFA76
:1038AC008A068B0790004E12001EE599F090078651
:1038BC0012000E900786E0FEA3E0FF74026F4E70BC
:1038CC000C1200C9851599751400751300023A6E17
:1038DC00900786E0FEA3E0FF90004E12001EE599D3
:1038EC00F090078612000E900786E0FEA3E0FFAC76
:1038FC000DAD0E8F028E038C068D07903EEF1200DD
:10390C002EE493F9740193FEEAD39EEB994009855A
:10391C001599751400751300023A6E900786E0FE37
:10392C00A3E0FF90004E12001EE599F0900786125E
:10393C00000E900786E0FEA3E0FFEFB40006EEB4A5
:10394C0001028003023A6E75FFA090001CE0D39434
:10395C00C7400B90001CE0C394C8F516801A900069
:10396C001CE0D39463400B90001CE0C39464F516E8
:10397C00800690001CE0F516E51675F002A4FFAE6B
:10398C00F08F6BEF90004E124409EFFCE0FDEC90D1
:10399C000051124409EDFCE0FDEC2DB5160280033C
:1039AC00023A600FEF90004E124409E56BFFE0FC09
:1039BC00EF900052124409ECFFE0FCEFC39CB516EB
:1039CC00028003023A60E56B900050124409E56BEB
:1039DC00FFE0FCEF900053124409ECFFE0FCEF2CED
:1039EC00B51671E56B900054124409E0C39516901E
:1039FC00079DF0E56B900055124409E0C3951690B5
:103A0C00079EF0E56B900058124409E0C3951690A0
:103A1C00079FF0E56B900059124409E0C39516908E
:103A2C0007A0F0E56B90005A124409E0C39516907C
:103A3C0007A1F0E56B90005B124409E0C39516906A
:103A4C0007A2F0122B687599F97518647517001296
:103A5C002B2480FE7599FF751864751700122B24A2
:023A6C0080FEDA
:093E600002387E0238DC02392729
:103A6E0022E513903E69F8282873023BAF90078633
:103A7E00E0FEA3E0FF90001212001EE0F599900701
:103A8E008612000E900786E0FEA3E0FF74116F4EC3
:103A9E007003751300023BAF856299023BAF90072E
:103AAE0086E0FEA3E0FF90004E12001EE0F599EFB7
:103ABE00B40107EEB4070375130090078612000ECB
:073ACE00023BAF900787E007
:0F3E6900023A78023A7B023AA6023AAC023AD108
:103AD500903E8AF8282873852499023BA4852A9963
:103AE500023BA4854499023BA4854799023BA485E2
:103AF5005199023BA4856099023BA4855699023BE6
:103B0500A4855899023BA4756F00900069E0700682
:103B1500900068E060028016A2A44006E56F4404A8
:103B2500F56FA2A54006E56F4402F56F801A900077
:103B35004AE0B40106E56F4410F56F900049E0B422
:103B45000106E56F4420F56FA207B34006E56F4413
:103B550001F56FA20CB34006E56F4408F56F856F5C
:103B650099803CA212B340077599FAC2128017A238
:103B75000FB3400575990F800B900023E0F59990E0
:103B85000023E4F0C20F80178542998012854B9976
:0F3B9500800D85469980087599FC800375130093
:103E8A00023ADC023AE2023AE8023AEE023AF40272
:103E9A003AFA023B00023B06023B0C023B68023B39
:0D3EAA008D023B92023B97023B9C023BA124
:0B3BA40090078612000E8003120048FC
:033E7800023BAC5E
:103BAF002290006BE0B4010385241190006BE0B408
:103BBF000203852A1190006BE0B403038544119032
:103BCF00006BE0B4040385471190006BE0B405036C
:103BDF0085511190006BE0B4060385561190006B70
:103BEF00E0B4070385581190006CE0FE90006DE083
:103BFF00C39E5003023C8690006BE0D39404402C8C
:103C0F0090006CE0D39511500990006DE0C39511B1
:103C1F0050028002D20090006CE0D39511500990B1
:103C2F00006DE0C395115002C200804990006BE017
:103C3F00B4041890006DE0C395115002D2009000AB
:103C4F006CE0D395114002C200802A90006CE0C353
:103C5F009511500990006DE0D3951150028002D25A
:103C6F000090006CE0D39511500990006DE0C39562
:103C7F00115002C200807E90006BE0D39404402C60
:103C8F0090006CE0C39511400990006DE0D3951141
:103C9F0040028002C20090006CE0C3951140099071
:103CAF00006DE0D395114002D200804990006BE087
:103CBF00B4041890006CE0C395115002C20090003C
:103CCF006DE0D395114002D200802A90006CE0C3C2
:103CDF009511400990006DE0D395114002D20090EC
:103CEF00006CE0D39511400990006DE0C395114031
:103CFF00028002C2002290006EE0B40103852411FD
:103D0F0090006EE0B40203852A1190006EE0B403B8
:103D1F000385441190006EE0B404038547119000B1
:103D2F006EE0B4050385511190006EE0B406038573
:103D3F00561190006EE0B4070385581190006FE0A4
:103D4F00FE900070E0C39E5003023DDB90006EE0DA
:103D5F00D39404402C90006FE0D39511500990003C
:103D6F0070E0C3951150028002D20290006FE0D331
:103D7F0095115009900070E0C395115002C2028056
:103D8F004990006EE0B40418900070E0C395115094
:103D9F0002D20290006FE0D395114002C202802A36
:103DAF0090006FE0C395115009900070E0D395110A
:103DBF0050028002D20290006FE0D395115009900B
:103DCF000070E0C395115002C202807E90006EE039
:103DDF00D39404402C90006FE0C3951140099000DC
:103DEF0070E0D3951140028002C20290006FE0C3D1
:103DFF0095114009900070E0D395114002D20280D6
:103E0F004990006EE0B4041890006FE0C395115014
:103E1F0002C202900070E0D395114002D202802AB4
:103E2F0090006FE0C395114009900070E0D3951199
:103E3F004002D20290006FE0D395114009900070BC
:0B3E4F00E0C3951140028002C2022275
:094409002582F582500205832290
:10002E00EF2F500205832582F582E5833E2EF58360
:01003E00229F
:08000300C3EF9DFFEE9CFE22FD
:08003F000806B60002180622B3
:0D000E00A3E004F070061243FFE004F022AE
:08441B000816B6FF0218162274
:0E43E300048007C3CE13CECF13CFD5E0F62251
:1041FB00BC000FBE0008ED8FF084FFADF022E4FE93
:10420B00FF22BE000DEF60FE54F0606F20E703024B
:10421B0042B1EAC0E0EBC0E078017A0075F001EE44
:10422B0020E710EF25E0FFEE33FE0AC5F023C5F0C3
:10423B0030E7F0EA5407F9096A7A007B006001085D
:10424B00C3EC9E40167004ED9F4010ED9FFDEC9E5D
:10425B00FCE5F0CA4ACA03F5F08005E5F003F5F07A
:10426B00C3EE13FEEF13FFD9D77908CACBCAD8D048
:10427B00EAFEEBFFD0E0FBD0E0FA22EC8FF084FCFF
:10428B00ED54F045F0C48FF084FEEDC454F045F0CE
:10429B00C48FF084FDEEC4FE54F02DFFEE540F3CA2
:1042AB00FEADF07C0022790078008FF0EC7E0820C8
:1042BB00E70DC3CD33CD33C933C9C833C8DEF08462
:1042CB0049F9E5F08FF0BE00E6FD7C00E9FFE8FE62
:0142DB0022C0
:0E43F100F88FF0A4FFE5F0CE88F0A42EFE2297
:1043C300600D782B0243CD007830D8FED5E0F8227B
:1043D300EEC0E07E001241FBEFFDEEFCD0E0FE22DA
:03000B000243723B
:03001B0002438D10
:03002B000243A8E5
:03000000024412A5
:0944120075817375D000020818D1
:0B001E00E5822FF582E5833EF583228A
:0A43FF000582D58202158315822283
:10437200C0E0C0F0C083C082C0D075D00012080D6A
:10438200D0D0D082D083D0F0D0E032C0E0C0F0C034
:1043920083C082C0D075D000120810D0D0D082D095
:1043A20083D0F0D0E032C0E0C0F0C083C082C0D081
:1043B20075D000120813D0D0D082D083D0F0D0E0D4
:0143C20032C8
:00000001FF
